:100000000C94E3050C94BD280C94EA280C940B0680
:100010000C940B060C940B060C940B060C940B061C
:100020000C940B060C940B060C94750C0C940B069C
:100030000C940B060C940B060C940B060C940B06FC
:100040000C9417290C940B060C94BF2C0C94FA2CCE
:100050000C940B060C940B060C940B060C940B06DC
:100060000C940B060C940B06341C3B1C3B1C341CE0
:100070003B1C3B1C3B1C3B1C3B1C3B1C3B1C3B1CC8
:100080003B1C3B1C3B1C3B1C3B1CA31B3B1C3B1C51
:100090003B1C3B1C3B1C061B3B1C3B1C3B1C3B1CDE
:1000A0003B1C3B1C3B1C3B1C3B1C3B1C3B1C3B1C98
:1000B0003B1C3B1C3B1CAF1BAF1BAF1BAF1BAF1B49
:1000C000AF1BAF1BAF1BAF1B3B1C3B1C3B1C3B1CAC
:1000D0003B1C3B1C0B1BAE1BAE1BAE1BAE1B3B1CD1
:1000E000C51BCD1BD51BDD1BE51BED1BF51BFD1B30
:1000F000071C111C1B1C251C521B121B3B1C3B1CF0
:100100003B1C3B1CA31B3B1C3B1C3B1C3B1C3B1CD0
:100110003B1C3B1C3B1CAD1BAD1BAD1BAD1B3B1C63
:10012000C51BCD1BD51BDD1BE51BED1BF51BFD1BEF
:10013000071C111C1B1C251C521B121B3B1C3B1CAF
:100140003B1C3B1CA31B456E746572206D656E7570
:100150002E2E2E00546F67676C6564206D69637284
:100160006F50504D00546F67676C656420696E7600
:1001700065727465642050504D2100546F67676C40
:100180006564205458206D7574696E672100546F42
:1001900067676C65642074656C656D657472792140
:1001A0000050726F746F636F6C206572726F722093
:1001B000776974682052580054696D656F757420B2
:1001C0007768656E20636F6E6E656374696E672015
:1001D000746F20525800507265737320616E7920DD
:1001E0006B657920746F2063616E63656C00436F8B
:1001F0006E6E656374696E6720746F2052582C2090
:10020000706F776572207570207468652052582071
:1002100028776974682062696E6420706C75672045
:100220006966206E6F74207573696E6720616C77E4
:100230006179732062696E642900546F67676C6529
:10024000642027696D6D656469617465206F7574DC
:100250007075742700546F67676C65642027736C32
:10026000617665206D6F64652700546F67676C6504
:10027000642027616C776179732062696E6427005E
:10028000546F67676C65642050504D206368616EE1
:100290006E656C206C696D697400536574205253EF
:1002A000534920696E6A656374696F6E2063686183
:1002B0006E6E656C2028303D3D64697361626C65CB
:1002C00029005365742050504D206D696E696D751D
:1002D0006D2073796E630053657420626561636F8E
:1002E0006E20696E74657276616C0053657420626D
:1002F0006561636F6E2064656C617900536574207D
:10030000626561636F6E206672657175656E637993
:1003100020696E20487A3A20303D64697361626CCE
:10032000652C2050783D504D52206368616E6E659B
:100330006C20782C2046783D465253206368616ECD
:100340006E656C2078005365742050574D2073748F
:100350006F702064656C6179202830206469736156
:10036000626C65642C20312D323535203D3D2030C6
:100370002E3173202D2035306D696E290053657440
:100380002050504D2073746F702064656C6179202B
:1003900028302064697361626C65642C20312D32D1
:1003A0003535203D3D20302E3173202D2035306DE8
:1003B000696E2900536574206661696C73616665B6
:1003C0002064656C61792028302064697361626CF7
:1003D00065642C20312D323535203D3D20302E31C5
:1003E00073202D2035306D696E29002A2A2A2A2A89
:1003F0002A2A2A2A2A2A2A2A2A2A2A2A2A2A2A2A5D
:100400002A2A2A2A2A2A2A2A0052582041636B655E
:1004100064202D2072657665727420737563636540
:10042000737366756C21002A2A2A2A2A2A2A2A2A04
:100430002A2A2A2A2A2A2A2A2A2A2A2A2A2A2A2A1C
:100440002A2A2A2A002A2A2A2A2A2A2A2A2A2A2A36
:100450002A2A2A2A2A2A2A2A2A2A2A2A2A2A2A2AFC
:100460002A2A0052582041636B6564202D20757044
:1004700064617465207375636365737366756C215D
:10048000002A2A2A2A2A2A2A2A2A2A2A2A2A2A2AF6
:100490002A2A2A2A2A2A2A2A2A2A2A2A2A2A0056BA
:1004A000616C69642063686F69636573206172655C
:1004B0003A205B315D2D5B31365D20286368616ECB
:1004C0006E656C20312D31362900536574206F75AF
:1004D0007470757420666F7220706F727420005B88
:1004E000585D2061626F7274206368616E67657326
:1004F00020616E64206578697420525820636F6EA5
:10050000666967005B535D2073617665207365746F
:1005100074696E677320746F205258005B525D20BF
:100520007265766572742052582073657474696EB2
:10053000677320746F2064656661756C7473005511
:100540007365206E756D62657273205B312D445D3D
:1005500020746F206564697420706F727473205BFF
:10056000452D515D20666F722073657474696E67E6
:100570007300202D20726563656976657220636F54
:100580006E666967757261746F722C207278207361
:100590007720000A0A6F70656E4C52536E67200018
:1005A0005365742073657269616C20626175647251
:1005B0006174653A200056616C69642063686F69F4
:1005C0006365733A2031202D20342B34202F2032C4
:1005D000202D2038202F2033202D20382B34202F81
:1005E0002034202D203132202F2035202D20313273
:1005F0002B34202F2036202D2031360053657420D7
:100600004368616E6E656C20636F6E6669673A2041
:1006100000536574204461746172617465202830F0
:100620002D32293A200053657420486F702063688A
:10063000616E6E656C7320286D61782032342C20D9
:1006400073657061726174656420627920636F6D97
:100650006D6173292076616C69642076616C7565C3
:100660007320312D3235353A20005365742063688C
:10067000616E6E656C2073706163696E67202878A7
:1006800031306B487A293A20005365742052462055
:10069000706F7765722028302D37293A2000536516
:1006A00074205246206D6167696320286865782947
:1006B00020652E672E203078444541444630304432
:1006C0003A2000536574206261736520667265711B
:1006D00075656E63792028696E20487A293A200072
:1006E0005B5A5D20656E746572207265636569761C
:1006F000657220636F6E66696775726174696F6E8B
:10070000207574696C79005B465D20646973706C58
:1007100061792061637475616C20667265717565BD
:100720006E636965732075736564005B525D206359
:10073000616C63756C6174652072616E646F6D20AD
:100740006B657920616E6420686F70206C697374CA
:10075000005B495D207265696E697469616C697AD4
:10076000652073657474696E677320746F20736B92
:10077000657463682064656661756C7473005B58AA
:100780005D20726576657274206368616E6765735B
:1007900020616E642065786974206D656E75005BFC
:1007A000535D20736176652073657474696E677339
:1007B00020746F20454550524F4D20616E64206576
:1007C000786974206D656E7500557365206E756D62
:1007D00062657273205B302D395D20746F20656413
:1007E000697420706172616D657465727300202D8B
:1007F0002053797374656D20636F6E6669677572D7
:100800006174696F6E000A0A6F70656E4C52536EA8
:100810006720005129204F757470757420626566D9
:100820006F7265206C696E6B20283D465329203A13
:100830002000502920536C617665206D6F6465201F
:10084000286578706572696D656E74616C293A20EF
:10085000004F292054696D65642042494E4420614F
:1008600074207374617274757020203A20004E29D0
:100870002050504D206F7574707574206C696D69CF
:1008800074656420202020203A20004449534142CE
:100890004C4544004D292050504D2052535349207F
:1008A000746F206368616E6E656C202020203A2092
:1008B000004C292050504D206D696E696D756D207A
:1008C00073796E63202875732920203A20004449EB
:1008D0005341424C4544004B29204661696C736189
:1008E000666520626561636F6E20696E74762E2086
:1008F00028312D32353573293A20004A29204661A6
:10090000696C7361666520626561636F6E20646502
:100910006C61792028302D323535203D3E20313034
:1009200073202D203135306D696E293A2000492918
:10093000204661696C7361666520626561636F6EF4
:10094000206672712E203A200048292050574D20F1
:1009500073746F702064656C6179202020202020E2
:10096000203A200047292050504D2073746F70208A
:1009700064656C6179202020202020203A200046E8
:1009800029204661696C736166652064656C6179D4
:10099000202020202020203A200050574D2063683E
:1009A000616E6E656C200066756E6374696F6E3A79
:1009B00020002920706F727420004454462055484E
:1009C000462033322D6269742031306368004F70E5
:1009D000656E4C52536E675258206D696E692034B3
:1009E0002F36636800466C7974726F6E2F4F726198
:1009F0006E67655258205548462038636800525843
:100A000020747970653A200044697361626C656492
:100A100000487A00203D3D200043616C63756C61A5
:100A2000746564207061636B657420696E746572AF
:100A300076616C3A20004229204D6963726F20284C
:100A400068616C66292050504D202020203A0041DA
:100A50002920496E7665727465642050504D206976
:100A60006E20202020203A003029204D757465200A
:100A700062757A7A657220286D6F73746C79293A81
:100A80000039292053657269616C20626175647256
:100A90006174653A00736D617274506F72740046D0
:100AA00072536B79005472616E73706172656E740B
:100AB0000044697361626C65640038292054656C78
:100AC000656D657472793A2020202020202000373F
:100AD00029204368616E6E656C20636F6E6669677E
:100AE0003A202000362920446174617261746520C7
:100AF00028302D32293A20202000352920486F70D7
:100B0000206368616E6E656C733A2020202020009F
:100B10003429204368616E6E656C2073706163696F
:100B20006E673A202000332920524620706F776587
:100B3000722028302D37293A2020200032292052D7
:100B400046206D616769633A202020202020202004
:100B500020003129204261736520667265717565D8
:100B60006E63793A20202000000000002400270056
:100B70002A0000000000250028002B0000000000D3
:100B800023002600290004040404040404040202CF
:100B900002020202030303030303010204081020FC
:100BA0004080010204081020010204081020000007
:100BB000000700020100000304060000000000001E
:100BC00000000D0FB32E11241FBECFEFD8E0DEBF03
:100BD000CDBF13E0A0E0B1E0E8EAFFE502C0059078
:100BE0000D92AA3FB107D9F716E0AAEFB3E001C012
:100BF0001D92A33AB107E1F71BE0C6ECDBE004C0AD
:100C00002297FE010E948C2FC23CD107C9F70E9497
:100C1000F82E0C94D22F0C940000A0E0B0E0E3E199
:100C2000F6E00C94A32FEC01A880B980CA80DB8089
:100C3000A114B104C104D10441F484E2A82E89EDC9
:100C4000B82E8BE5C82E87E0D82EC601B5012DE160
:100C500033EF41E050E00E945B2F27EA31E440E0AF
:100C600050E00E94072F7B018C01C601B5012DE1E8
:100C700033EF41E050E00E945B2FCA01B9012CEE36
:100C800034EF4FEF5FEF0E94072F6E0D7F1D801F27
:100C9000911F97FF04C06150704080409048688366
:100CA00079838A839B839B01AC015F77B901CA0179
:100CB000CDB7DEB7EAE00C94BF2F0E940D06089571
:100CC00084E193E00E940D060895609314037093ED
:100CD000150380931603909317030895A0E0B0E0E6
:100CE000E4E7F6E00C949C2FEC012B016A016115FE
:100CF000710519F0FB0191838083C114D10449F07F
:100D0000C6010297839728F020E030E040E050E0F1
:100D1000DCC0A9908A2D90E00E94902F892BC9F702
:100D2000FDE2AF1621F4A9903324339405C08BE281
:100D3000A81609F4A9903324C114D10421F0E0E1EC
:100D4000CE16D10411F5F0E3AF1669F48881883727
:100D500011F0883541F4A980229682E0382A20E1FA
:100D6000C22ED12C12C0C114D10479F4E0E3AE1626
:100D700059F199E9E92E99E9F92E99E9092F99E1B3
:100D8000192F8AE0C82ED12C3AC0FAE0CF16D10430
:100D900091F080E1C816D10429F0E8E0CE16D10424
:100DA000F9F415C0BFEFEB2EBFEFFB2EBFEF0B2FFB
:100DB000BFE01B2F24C0A9E9EA2EA9E9FA2EA9E970
:100DC0000A2FA9E11A2F1BC0F8E0CF2ED12CEFEF8C
:100DD000EE2EEFEFFE2EEFEF0E2FEFE11E2F0FC0E6
:100DE0009601442737FD4095542F6FEF7FEF8FEF2B
:100DF0009FEF0E94392FC901DA017C018D0120E0AB
:100E000030E040E050E060E03601882477FC8094D8
:100E1000982C70EDB72EBA0CF9E0FB1570F48A2D02
:100E200081548A3118F499ECB92E06C08A2D815666
:100E30008A3148F589EAB82EBA0C8B2D90E08C15D2
:100E40009D050CF56F3FE9F0E216F3060407150760
:100E5000B8F0CA01B901A40193010E94072F9B01B8
:100E6000AC018B2D90E0A0E0B0E0280F391F4A1FA5
:100E70005B1F281739074A075B0710F061E001C0C4
:100E80006FEFA990C6CF4114510451F0662311F0C1
:100E9000219703C031FE04C02297F201D183C083A1
:100EA00030FE07C050954095309521953F4F4F4FEC
:100EB0005F4F67FF0AC082E290E09093A2068093A2
:100EC000A1062FEF3FEF4FEF5FEFB901CA01CDB79A
:100ED000DEB7E1E10C94B82FFC0188279927E8944C
:100EE00021912032E9F3293010F02E30C8F32B3253
:100EF00041F02D3239F4689404C00E94C107820F7A
:100F0000911D219120532A30C0F31EF490958195B4
:100F10009F4F08954AEF53E00E948F07089500976E
:100F200031F4DA018D919C91009709F40EC0DC0137
:100F3000FB013D912191222319F03217C9F3FACF19
:100F4000332331F4DA011D921C92882799270895E2
:100F50001197AF93BF93FB013D912191321771F42B
:100F6000332321F488279927119702C01E921196E6
:100F7000FA01A193B0839F918F910895222369F77D
:100F8000EACF7AE0979F902D879F802D910D1124B5
:100F900008958091FC03813019F482E08093FC0372
:100FA0008091FC03833019F484E08093FC0308955E
:100FB00080912604E82FF0E03496DF0126E0AA0FA6
:100FC000BB1F2A95E1F720E030E040E050E060E010
:100FD00070E0F999FECFCB018A0F9B1F92BD81BDB6
:100FE000F89A80B5542F432F322F2227280F311D16
:100FF000411D511D6F5F7F4F6430710551F72E51B8
:101000003E4B414C5E4D19F020E030E01FC09F0187
:1010100086E0220F331F8A95E1F72C5F3F4FEDEFFB
:10102000F3E0F999FECF32BD21BDF89A80B58193E6
:101030002F5F3F4F84E0E632F80799F720E030E079
:101040008091FD03893011F421E030E0C901089559
:1010500089E08093FD0380E092ECA1E0B0E0809312
:10106000FE039093FF03A0930004B093010487E074
:1010700080930A0480EC92E9ADEEB9E1809302041A
:1010800090930304A0930404B093050485E0809337
:101090000B048DEE9EEFADEABEED809306049093B7
:1010A0000704A0930804B0930904ACE0B4E080E026
:1010B00090E0863010F0E0E004C0FC01ED51FC4F00
:1010C000E081ED9301968831910599F782E0809354
:1010D00024048AE08093250408958436910520F441
:1010E000BC0180E090E025C08E3B910550F48A550C
:1010F0009040BC0180E090E02AE030E040E050E029
:1011000016C0823D910550F4845B9040BC0180E0A4
:1011100090E024E630E040E050E009C08D5C904073
:10112000BC0180E090E028E532E040E050E00E9421
:10113000072F24E630E040E050E00E94072F08959A
:1011400090E08C599F4F0E946D080895DC0198969D
:10115000EC91F0E0E770F070E552FC4F808108956B
:101160008F929F92AF92BF92CF92DF92EF92FF92B7
:101170000F931F938C010E94A608D80197962C917B
:1011800030E043E150E0249FF001259FF00D349FB3
:10119000F00D1124E85EFC4F80809180A280B38026
:1011A00090E00F96AA2797FDA095BA2FBC01CD011C
:1011B00020E43FE14DE750E00E94072FA501940194
:1011C0000E94392F69017A0180ED97E0A0E0B0E03C
:1011D000C80ED91EEA1EFB1ED80198968C91887104
:1011E00081F060E07EEE8AEB9BE0A50194010E9415
:1011F000392F28513C4F4F4F5F4FC20ED31EE41E74
:10120000F51E87EE93E0A0E0B0E0C80ED91EEA1EFE
:10121000FB1EC701B60128EE33E040E050E00E941B
:10122000392FCA01B90128EE33E040E050E00E94B6
:10123000072F1F910F91FF90EF90DF90CF90BF90FD
:10124000AF909F908F9008958F3F910509F010F413
:1012500080E0089522E08030920710F481E0089544
:101260008050934010F083E0089582E00895CF927B
:10127000DF92FF920F931F93CF93DF93F82FEB0131
:101280006A01182F1695E0E088819981D6018C9328
:101290008A819B8111968C9311978C819D811296E6
:1012A0008C9312978E819F8113968C93139728812C
:1012B00039814A815B816C817D818E819F8192958C
:1012C000990F990F907C832F8370982B852F8370B3
:1012D000880F880F982B872F83708295807F982B9B
:1012E00014969C9385E090E0C80ED91E2896EF5F77
:1012F0001E1750F6F0FF21C0888199810E942409B1
:10130000F82E8A819B810E942409182F8C819D814F
:101310000E942409082F8E819F810E942409F29443
:10132000FF0CFF0C50ECF5221295107F1F29182B93
:10133000000F000F012BD6010C93DF91CF911F916D
:101340000F91FF90DF90CF90089523E080329207B5
:1013500018F420E030E026C023E0883E920748F4ED
:101360009C012F513340F4E036952795FA95E1F72B
:1013700019C027E0803D920720F49C012C5D33408A
:1013800011C028E08839920718F02FEF33E00AC027
:101390009C01285C3740E4E036952795EA95E1F713
:1013A0002D503C4FC90108959C0136952795257510
:1013B0003575821B930B9C0136952795369527959D
:1013C0002373337383739373280F391FC90144E068
:1013D000969587954A95E1F7820F931F8F709F70BE
:1013E00021E031E0AC01429FC001439F900D529F2C
:1013F000900D1124892F0895382F20E08091E80561
:101400009091E9058227932740E061E270E19C0119
:10141000220F331F97FF04C0C9018627972701C0F9
:10142000C9014F5F483099F79093E9058093E8052B
:101430000895882339F02D9800002B9A00002D9AEA
:10144000000008952D9800002B9800002D9A0000B0
:1014500008952D9A000083B12D98000090E0F4E0EB
:1014600096958795FA95E1F7817008950F931F93EC
:10147000082F5C9A2D985C9810E0802F80780E944D
:10148000190A000F1F5F1830C1F72D981F910F9197
:1014900008958F770E94360A08950F931F93082F9F
:1014A00010E0802F80780E94190A000F1F5F18300B
:1014B000C1F72D981F910F9108950F931F932D98A9
:1014C00080E000E0182F110F0E94290A810F0F5FA2
:1014D0000830C1F71F910F9108950E94490A0E9498
:1014E0005D0A5C9A08951F93162F80680E94360A41
:1014F000812F0E944D0A5C9A1F9108951F931091AD
:1015000006041827EDEFF3E0E80FF11D89E7678582
:101510000E94730A8DE3612F0E94730A82E4612F97
:101520000E94730A1F91089586E20E946D0A089531
:101530000F931F938C018CE1F80164810E94730A60
:101540008DE1F80165810E94730A8EE1F8016681E0
:101550000E94730A80E2F80167810E94730A81E2A7
:10156000F80160850E94730A82E2F80161850E9499
:10157000730A83E2F80162850E94730A84E2F8012B
:1015800063850E94730A85E2F80164850E94730AEC
:101590008AE2F80165850E94730A8EE6F801668585
:1015A0000E94730A8FE6F80167850E94730A80E73C
:1015B000F80160890E94730A81E7F80161890E943D
:1015C000730A82E7F80162890E94730A1F910F91E2
:1015D0000895EF92FF920F931F93CF93DF937B01B8
:1015E0008C01603028E372072CE982072CE1920716
:1015F00028F520E836E948E950E00E94392FE90152
:101600006897B90180E090E020E839E647E65FEFAF
:101610000E94072F6E0D7F1D801F911F02E0660F35
:10162000771F881F991F0A95D1F721E732E040E024
:1016300050E00E94392F890180E421C020E03DE282
:1016400041E351E00E94392FE9016897B90180E038
:1016500090E020E033ED4EEC5EEF0E94072F6E0D20
:101660007F1D801F911F660F771F881F991F21E71D
:1016700032E040E050E00E94392F890180E69E016F
:101680002F71622F680F85E70E94730A86E7612F2A
:101690000E94730A87E7602F0E94730ADF91CF913F
:1016A0001F910F91FF90EF9008959F92AF92BF927C
:1016B000CF92DF920F93DF93CF9300D000D0CDB7BE
:1016C000DEB7982E83E00E946D0A8093420484E086
:1016D0000E946D0A8093430486E060E00E94730AD2
:1016E00087E061E00E94730A89E06FE70E94730A55
:1016F0008AE065E00E94730A8BE062E10E94730A4F
:101700008CE065E10E94730A8DE06DEF0E94730A20
:101710008EE060E00E94730A992019F087E793E059
:1017200008C08091240423E1829FC0011124885EB7
:101730009C4F0E94980A80E36CE80E94730A82E33F
:101740006FE00E94730A83E362E40E94730A84E3F9
:101750006AE00E94730A85E36AE20E94730A86E3E4
:101760006DE20E94730A87E364ED0E94730A88E3C6
:1017700060E00E94730A89E360E00E94730A992086
:1017800049F02EE1A22E2EEBB22E21ECC22E2EED30
:10179000D22E08C0A0900604B0900704C0900804A0
:1017A000D09009040AE38D2D9927AA27BB278983A6
:1017B0009A83AB83BC83802F69810E94730A802F38
:1017C0008B5F69810E94730ADC2CCB2CBA2CAA2473
:1017D0000F5F0E3341F783E46FEF0E94730A84E4D6
:1017E0006FEF0E94730A85E46FEF0E94730A86E42C
:1017F0006FEF0E94730A992019F08DE666E003C02E
:101800008DE660910A040E94730A89E760E00E94F5
:10181000730A8AE760910B040E94730A83E760E011
:101820000E94730A84E760E00E94730A992029F0FD
:1018300060EC72E98DEE99E108C06091020470914C
:10184000030480910404909105040E94E90A0F901A
:101850000F900F900F90CF91DF910F91DF90CF906D
:10186000BF90AF909F90089587E061E00E94730A57
:101870008EE764E20E94730A88E063E00E94730AC4
:1018800088E060E00E94730A87E065E00E94730AC6
:1018900085E062E00E94730A83E00E946D0A8093F3
:1018A000420484E00E946D0A809343040895582FF7
:1018B00040915305842F90E0FC01EF70F0709F0180
:1018C0002F5F3F4F64E0959587956A95E1F728175C
:1018D000390751F0ED5BFA4F5083842F8F5F8F7083
:1018E000407F842B8093530508951F920F920FB66B
:1018F0000F9211241F932F933F934F935F936F93F6
:101900007F938F939F93AF93BF93CF93DF93EF9387
:10191000FF93C0918600D09187002091950530916A
:10192000960580917405882309F047C0CE01821B7B
:10193000930B9C018091250487FD02C03695279565
:1019400099E0253C390708F18091AA038630D0F050
:101950008091AA038F3FB1F020E00EC0E22FF0E0AB
:10196000EE0FFF1FDF01AB58BA4F8D919C91E657E8
:10197000FC4F918380832F5F8091AA03281770F317
:10198000109273051092AA0318C082E02D3B38070D
:1019900060F18091AA03803140F51091AA03C9013A
:1019A0000E94A509E12FF0E0EE0FFF1FEB58FA4F60
:1019B000918380831F5F1093AA03D0939605C093F1
:1019C0009505FF91EF91DF91CF91BF91AF919F91DD
:1019D0008F917F916F915F914F913F912F911F91C7
:1019E0000F900FBE0F901F9018958FEF8093AA0352
:1019F000E4CF83E0809380008AE980938100809126
:101A0000250486FD05C0809181008064809381005B
:101A10008FEF9FEF909389008093880080916F00F3
:101A2000806280936F0008956F3020F086958695D0
:101A3000805408958DE0689F802D11240895982F7B
:101A40008091E105882329F4933009F043C081E0B7
:101A500005C0813049F4913021F482E08093E105A2
:101A600008951092E1050895803190F5E82FF0E097
:101A7000EB58FA4F90838F5F8093E105803151F5E9
:101A800020917405A7E7B5E0213039F41196EC9167
:101A90001197E695E6958C9109C08D919C911197CF
:101AA000E92FE695E695E69596958795E03140F421
:101AB000F0E090E0EE0FFF1FE657FC4F918380832C
:101AC00010927305129685E0A538B807E9F60895D7
:101AD0001092E10508950F931F93CF93DF93909198
:101AE000E105992339F48F3009F002C181E0809338
:101AF000E105FEC0983148F4E92FF0E0EC58FA4FC8
:101B000080839F5F9093E105F3C0983109F0EEC0A8
:101B1000882309F0EBC0C0E0D0E00BE010E0DE016C
:101B200063E0AA0FBB1F6A95E1F7C09FB001C19F98
:101B3000700DD09F700D1124FB01EB58FA4F80817E
:101B40002181922F977095958795FD01EE0FFF1FCC
:101B5000E657FC4F91838083FB01EA58FA4F3081AE
:101B60003695369536952181422F4295440F407E19
:101B7000842F832B269526952695922F97709595E1
:101B80008795FD01EE0FFF1FE457FC4F9183808383
:101B9000FB01E958FA4F808182958695869583707E
:101BA0004181942F990F990F292F282B4295469503
:101BB0004695437082818170880F880F382F342BAF
:101BC00035952795FD01EE0FFF1FE257FC4F31833E
:101BD0002083FB01E758FA4F308136952181422F4F
:101BE000479544274795842F832B2695922F9770EE
:101BF00095958795FD01EE0FFF1FE057FC4F9183F0
:101C00008083FB01E658FA4F308132953F70218185
:101C1000422F4295407F842F832B22952F70922F45
:101C2000977095958795FD01EE0FFF1FEE56FC4FBF
:101C300091838083FB01E558FA4F8081881F8827B4
:101C4000881F4181942F990F292F282B441F442747
:101C5000441F82818370880F382F342B3595279548
:101C6000FD01EE0FFF1FEC56FC4F31832083FB017B
:101C7000E358FA4F3081369536952181422F4295AF
:101C8000440F440F407C842F832B26952695922F5A
:101C9000977095958795AA0FBB1FFD01EA56FC4FDB
:101CA0009183808362587A4FFB012081229526958B
:101CB00027704181342F330F330F330F832F822B43
:101CC000942F92959695977095958795A856BC4FA9
:101CD00011969C938E932196C230D10509F01FCFA7
:101CE00080918B0583FD02C0109273051092E1056F
:101CF000DF91CF911F910F910895DF92EF92FF92A4
:101D00000F931F93CF93DF93682F4091E1054423F6
:101D100059F4883AB1F41092E9051092E80588EA7E
:101D20000E94FC0981E06FC0413019F48093E60500
:101D300004C0423031F48093E705862F0E94FC09ED
:101D40005DC07091E705272F30E0220F331FE42F8D
:101D5000F0E0C90102968E179F0734F0433268F70E
:101D6000EE58FA4F6083E9CF2D5F3F4F4091E80571
:101D70005091E905E217F30749F4962F80E04827D0
:101D800059275093E9054093E80538C0862F90E025
:101D90004817590789F58091E605813069F5713159
:101DA00018F080E18093E705D090E705F5E7EF2E86
:101DB000F5E0FF2E00E010E01BC0F701D081C0E08D
:101DC000818190E08C2B9D2BE3E096958795EA9599
:101DD000E1F70E94A509F801EE0FFF1FE657FC4F3F
:101DE000918380830F5F1F4F82E090E0E80EF91E21
:101DF0000D1518F3109273051092E1058091E1051D
:101E0000882319F08F5F8093E105DF91CF911F91B7
:101E10000F91FF90EF90DF90089510924A04109276
:101E20004F0410924E0410925104109250040895E1
:101E3000882319F460E071E002C063E071E08FE78D
:101E400096E00E94AA2C0895CF92DF92EF92FF9223
:101E50001F93182F0E946D299B01AC018091E20510
:101E60009091E305A091E405B091E50569017A013F
:101E7000C81AD90AEA0AFB0AD701C6018958934150
:101E8000A040B04010F01092E1052093E20530939D
:101E9000E3054093E4055093E50590917405892F7F
:101EA0008150823020F4812F0E941F0D0BC093308F
:101EB00021F4812F0E946B0D05C0943019F4812FFD
:101EC0000E947D0E1F91FF90EF90DF90CF900895BC
:101ED000FF920F931F93CF93DF93182F092FF62EA6
:101EE0008EE30E94730A212F302FC901EC0110E00C
:101EF00005C08FE769910E94730A1F5F1F15C8F321
:101F000085E064E00E94730A83E00E946D0A80937A
:101F1000420484E00E946D0A809343040E946D296C
:101F2000609344047093450480934604909347045F
:101F300087E069E00E94730A81E08093FC03DF91EF
:101F4000CF911F910F91FF9008950E94680F80918B
:101F5000FC038130D9F40E946D2920914404309112
:101F600045044091460450914704621B730B840B57
:101F7000950B605A76488140904040F4E8CF8FE757
:101F800096E067E071E00E94AA2C08958091FC031E
:101F90008130A9F308958FE796E06EE70E94732ED3
:101FA0000895BF92CF92DF92EF92FF920F931F930B
:101FB000CF93DF936C018FE796E06EE70E94732E5C
:101FC000760100E010E0C0E0D0E080E2B82E0AC068
:101FD0000830110521F49E012095F6012087089410
:101FE000E11CF11CF7016081862F8D57823040F48F
:101FF0008FE796E06DE70E94732EF70160816B25F5
:102000008FE796E00E94732E0115110551F0F7013C
:1020100080819E01280F311DC32FDD27C20FD31FE2
:10202000D0700F5F1F4F0930110591F6DF91CF91EE
:102030001F910F91FF90EF90DF90CF90BF90089588
:10204000DF93CF93CDB7DEB729970FB6F894DEBFF5
:102050000FBECDBF382FE62F8091580590E0019636
:1020600064E270E00E94262F982F8093580588E93B
:10207000898380E18A83913071F0913028F0923029
:1020800099F09330E1F416C085E08B8381EF8C8367
:102090002F5F2D8317C09B8381EF8C8384E6489F3D
:1020A000C00111249D830EC084E08B8381EF8C835B
:1020B0003D8308C09B8381EF8C83ED8303C00E9426
:1020C000CB0F04C0CE0101960E94D10F29960FB606
:1020D000F894DEBF0FBECDBFCF91DF9108950F936F
:1020E0001F93CF93DF93182F092F8FE796E06EE7AA
:1020F0000E94732E212F302FC901EC0110E000E265
:1021000088818D57823040F48FE796E06DE70E941A
:10211000732E8881802788838FE796E069910E94DB
:10212000732E1F5F193061F78FE796E06EE70E940C
:10213000732EDF91CF911F910F910895DF93CF936D
:10214000CDB7DEB729970FB6F894DEBF0FBECDBF6F
:10215000382F80915805882379F48EEF89833A834C
:102160006B83842F90E0959587958C832D831986BA
:1021700018861F821E822FC040915305842F90E045
:102180009C012F70307054E0959587955A95E1F732
:102190008217930721F18DEF89831A821B82DE015A
:1021A000149620E008C0ED5BFA4F80818D93405F6C
:1021B0002F5F263069F0842F90E0FC0134E0F59524
:1021C000E7953A95E1F78F709070E817F90759F79E
:1021D000409353052A83CE0101960E946F1080918F
:1021E000580590E0019666E070E00E94262F8093EB
:1021F000580529960FB6F894DEBF0FBECDBFCF911C
:10220000DF9108959F92AF92BF92CF92DF92EF92AB
:10221000FF920F931F93B82EA62ED42EC22E902E6F
:102220000E946D297B018C0180914205209154050B
:102230003091550540915605509157058823B1F0CE
:10224000D801C701821B930BA40BB50B815E9E4284
:10225000A040B04020F12C2DDC1408F42D2D8B2D46
:102260006A2D422F292D0E94201011C0D801C701CC
:10227000821B930BA40BB50B81539547A040B04034
:1022800070F08B2D6A2D4D2D2C2D0E949E10E0920A
:102290005405F092550500935605109357051F916C
:1022A0000F91FF90EF90DF90CF90BF90AF909F90F5
:1022B0000895FF920F931F938C01F62E8FE796E0FF
:1022C0000E94732EF80184818F2584831F910F91C2
:1022D000FF900895FF920F931F938C01F72E0E9499
:1022E0005911C8016F2D0E9459111F910F91FF9034
:1022F0000895BF92CF92DF92EF92FF920F931F93B8
:102300007C01B62E6A010FE716E0C80165EB0E945A
:10231000732EC80162E60E94732EF7011482C70172
:102320006B2D0E945911C701B6010E946A111F91BD
:102330000F91FF90EF90DF90CF90BF9008958CE0C9
:1023400060E00E94F4298BE061E00E94F4298DE0B6
:1023500061E00E94F42982E060E00E94F42984E0B8
:1023600061E00E94F4290895EF92FF920F931F936A
:10237000009771F19C0140E050E068E478EE81E064
:1023800090E00E945B2FC901DA017C018D0183E19D
:1023900061E00E94602A8FEFE816F1040105110543
:1023A00039F030F0EFEFEE2EF12C012D112D0AC097
:1023B000E114F1040105110529F471E0E72EF12C77
:1023C000012D112DE092B3008091B000806107C013
:1023D00083E160E00E94602A8091B0008F7E80934C
:1023E000B0001F910F91FF90EF90089583E161E09D
:1023F0000E94F42983E160E00E94602A82E08093D9
:10240000B00085E08093B10083E061E00E94F42990
:1024100083E060E00E94602A08951F93182F0E94B5
:102420006D296093540570935505809356059093DC
:10243000570510934205112329F440E855E260E066
:1024400070E004C040E051EE60E070E08FE796E09D
:102450000E94792D1F910895AF92BF92CF92DF9283
:10246000EF92FF920F931F93DF93CF93CDB7DEB719
:102470006C970FB6F894DEBF0FBECDBF0E946D29DA
:102480007B018C0181E00E94550BB4E7AB2E6E01FD
:102490000894C11CD11CA3E0BA2EA982C60161E038
:1024A0000E94A50FB092FC030E94340C6AEF70E00A
:1024B00080E090E00E9493298091FC03833009F032
:1024C0008AC08FE796E00E94002E892B09F083C016
:1024D0000E946D296E197F09800B910B6058734C17
:1024E000894C914008F077C0D8CF8FE70E94490A05
:1024F0000E945D0A843509F05CC089830E945D0AF0
:10250000182F00E010934105009340050E945D0ADA
:10251000080F111D10934105009340050E945D0AAC
:1025200080933F050E945D0A80933E05813108F04B
:1025300040C0FF2407C00E945D0A025E1A4FF801E6
:102540008083F3940F2D10E080913E0590E0880F7A
:10255000991F0817190778F380E78983CE01019640
:1025600061E00E94A50F83E08093FC030E94340C7D
:1025700062E370E080E090E00E9493298091FC0388
:102580008330A9F08FE70E94490A0E945D0A8035D6
:1025900081F4898307E214E00E945D0AF8018193C7
:1025A0008F01F4E002341F07B9F781E003C082E035
:1025B00001C083E06C960FB6F894DEBF0FBECDBFAE
:1025C000CF91DF911F910F91FF90EF90DF90CF900F
:1025D000BF90AF9008958091FC03833009F085CFC0
:1025E000E6CF83E00E946D0A8093420484E00E945B
:1025F0006D0A8093430487E061E00E94730A6AE0F9
:1026000070E080E090E00E9493290E94340C00006A
:1026100008950F931F93082F19C05E9A409A64E69D
:1026200070E080E090E00E9493295E98409864E614
:1026300070E080E090E00E9493291F5F101768F31C
:102640006CE271E080E090E00E94932910E0F6CF08
:10265000482F392F25E00DC0F999FECF1FBA842FDE
:10266000932F92BD81BD60BD0FB6F894FA9AF99A86
:102670000FBE215059F0F999FECF842F932F92BDB0
:1026800081BDF89A80B5681739F7089582E00E94F5
:1026900009130895CF92DF92EF92FF920F931F9349
:1026A000CF93DF93C0E0D0E008E110E03EE1C32E1D
:1026B0003EEBD32E31ECE32E3EEDF32E809126043B
:1026C00090E0049626E0880F991F2A95E1F7A7016C
:1026D0009601002E04C056954795379527950A9484
:1026E000D2F78C0F9D1F622F0E942813219608504D
:1026F0001040C430D10511F7C0E0D0E0809126042D
:1027000090E016E0880F991F1A95E1F78C5F9E4FB5
:10271000FE01E350FC4F8C0F9D1F60810E94281327
:102720002196C932D10551F7DF91CF911F910F91B9
:10273000FF90EF90DF90CF90089580E490E060915B
:1027400026040E9428130895F999FECF80E490E0B2
:1027500092BD81BDF89A80B580932604843020F024
:10276000109226040E949D1308951F93182F0E9413
:10277000A41380912604811731F0143020F41093B3
:1027800026040E949D131F91089580915A0581305F
:10279000D1F0813020F0823009F043C037C082E1AF
:1027A0000E94932A892B09F03CC081E080935A054E
:1027B0000E945F2960935B0570935C0580935D05C3
:1027C00090935E05089582E10E94932A892BD9F4A3
:1027D0000E945F2920915B0530915C0540915D0569
:1027E00050915E05621B730B840B950B695E734001
:1027F00080409040B0F082E080935A0580ED97E0F1
:102800000E94B411089510925A05089582E10E9421
:10281000932A892B31F080E090E00E94B41110924D
:102820005A050895AF92BF92CF92DF92EF92FF9236
:102830000F931F93CF93DF938CE00E946D0A882340
:10284000C9F58FE796E063E171E00E94AA2C5E9AD9
:10285000409A80E00E94550B0E94340C5E9840988C
:1028600029C080917405882339F08FE796E00E9493
:102870003A2E0E94240F1EC08091DF05C82FD0E0A1
:102880009E012F5F3F4F2F7130708091DE0590E0E9
:102890002817390779F08FE796E00E943A2ECB543B
:1028A000DA4F88838091DF0590E001968F719070F8
:1028B0008093DF058FE796E00E94002E892B89F632
:1028C0008091FC03843009F08CC00E946D296093D4
:1028D00063057093640580936505909366056115A3
:1028E00071058105910561F481E090E0A0E0B0E020
:1028F0008093630590936405A0936505B093660586
:1029000080916F0590917005816090937005809320
:102910006F0583E08093FC038FE70E94490ACCEAAD
:10292000D5E00E945D0A899305E0C53BD007C9F751
:10293000409197058091AC05282F30E0842F90E0DE
:102940008227932786FF40C080E44827409397055D
:10295000C90188739070C89709F510E014C01F5F13
:1029600080912504E12FF0E084FF06C0E455FA4F82
:1029700080810E94570C07C0E455FA4F8FE796E01C
:1029800060810E94732E212F30E08091AC0590E091
:10299000877090708217930714F716C02F733070EA
:1029A000232B91F48091AD05809367058091AE054E
:1029B000809369058091AF0580936A058091B20587
:1029C00080937105109272058091E005813019F4B1
:1029D00082E08093E0058091E005833011F410924D
:1029E000E0050E946D295B016C0180916B0590915F
:1029F0006C05A0916D05B0916E050097A105B1051C
:102A0000C9F0A6019501281B390B4A0B5B0BDA01B3
:102A1000C901885B9B40A040B04060F00E94940ACE
:102A20008093680510926B0510926C0510926D05ED
:102A300010926E058DEF93E00E94B00820915F0523
:102A400030916005409161055091620586017501E4
:102A5000E21AF30A040B150BE616F7060807190726
:102A600008F4EDC0A0925F05B0926005C0926105C8
:102A7000D092620580917305883008F0D7C08091AC
:102A800073058F5F80937305E0906305F090640594
:102A90000091650510916605E114F1040105110529
:102AA00011F18DEF93E00E94B008AE18BF08C00A84
:102AB000D10A6A157B058C059D0588F48091250453
:102AC00085FD04C080ED97E00E94B411109263056B
:102AD00010926405109265051092660504C080E0AE
:102AE00090E00E94B41190919705907C9093970587
:102AF0000091DF051091DE050117B1F18091E0052D
:102B0000823091F59058909397058DEF93E00E9455
:102B1000A608893010F048E002C0482F415030E04C
:102B200013C03F5FA32FB0E0812F90E0FC01EB5476
:102B3000FA4F2081FD01E956FA4F2083AB52BA4F7C
:102B40002C930196182F1F71341710F4101749F7A2
:102B50001093DE05832F895C90919705892B8093D4
:102B600097053093D5051AC02091E0052430D1F4A3
:102B70009091D505E6EDF5E0A8E9B5E0292F30E024
:102B80002E0F3F1F02C081918D93E217F307D9F7F3
:102B9000995C80919705982B9093970583E080939B
:102BA000E00525C080915A05823031F49160909300
:102BB00097055E9A409A10C0909397055E9840984A
:102BC000222319F481E08093E0058091E0058330B1
:102BD00019F484E08093E005F894809125048770CF
:102BE0006AE873E048E955E00E94370978945D9AF5
:102BF000419A809159050E947E0A8DEF93E00E94D0
:102C0000A608682F87E995E00E94680FE0915905B2
:102C1000EF5FE0935905E83131F0F0E0E350FC4F0D
:102C20008785882361F41092590509C08091730546
:102C3000883011F45E9A409A89E080937305809100
:102C40002504887171F18091FC03823051F58091E7
:102C50006F0590917005880F991F90937005809370
:102C60006F0583E08093FC030E94340C0E946D2961
:102C700060936B0570936C0580936D0590936E0562
:102C8000611571058105910561F481E090E0A0E096
:102C9000B0E080936B0590936C05A0936D05B093A5
:102CA0006E058091250484FF1EC080916F05909170
:102CB00070058E7F0E94D409182F8091670560915E
:102CC00071050E94140D082F80916805612F0E94E4
:102CD000140D282F8091690560916A05402F00919D
:102CE00026040E9402115D9841980E94C513DF914D
:102CF000CF911F910F91FF90EF90DF90CF90BF90F9
:102D0000AF90089510921C0585E6E7EBF4E0DF0133
:102D10001D928A95E9F708951F93182F8F3719F0A0
:102D2000883009F042C0E0911C05EE2309F45EC032
:102D3000E150E0931C05F0E0E954FB4F10828FE76F
:102D400096E06DE00E94732E10E00DC0E12FF0E0E0
:102D5000E954FB4F6081772767FD70958FE796E018
:102D60000E94732E1F5F80911C05181778F38FE760
:102D700096E060E20E94732E8FE796E06DE00E947D
:102D8000732E10E00DC0E12FF0E0E954FB4F60819D
:102D9000772767FD70958FE796E00E94732E1F5F7F
:102DA00080911C05181778F31FC08B3119F40E940D
:102DB000821622C08D3001F18A30F1F080911C051D
:102DC0008436A0F4612F772767FD70958FE796E032
:102DD0000E94732E80911C05E82FF0E0E954FB4F10
:102DE00010838F5F80931C0580E007C08FE796E01B
:102DF00067E00E94102BF8CF81E01F9108951F9388
:102E0000CF93DF93CCE0D4E010E03BC08FE796E0B7
:102E100062E271E00E94A72C8FE796E0612F4AE002
:102E200050E00E941E2C8FE796E06FE271E00E9456
:102E3000A72C699170E080E090E020910B0430E0D5
:102E400040E050E00E94072F20E137E240E050E0F0
:102E50000E94072FDC01CB01409102045091030432
:102E60006091040470910504480F591F6A1F7B1F6D
:102E70008FE796E02AE030E00E94E52B1F5F1831D3
:102E800019F08881882311F6DF91CF911F91089561
:102E9000EF92FF920F931F93882339F48FE796E008
:102EA00068E07AE00E942E2B3BC090E00E946D0803
:102EB00024E630E040E050E00E94392F122F032F2B
:102EC000F42EE52E622F732F842F952F2AE030E009
:102ED00040E050E00E94392F8FE796E0BA01A90147
:102EE0002AE030E00E94D62B8FE796E06EE20E9447
:102EF000102B612F702F8F2D9E2D2AE030E040E0A7
:102F000050E00E94392FAB01BC018FE796E02AE028
:102F100030E00E94D62B8FE796E063E70E94422BB9
:102F20001F910F91FF90EF900895FF920F931F93C1
:102F3000CF93DF938FE796E06EEF79E00E94ED2A62
:102F400080912704813041F48FE796E065EE79E0C7
:102F50000E942E2BFF2466C0823029F48FE796E072
:102F60006EEC79E0F5CF8430A9F78FE796E06AEB55
:102F700079E0EECFCF2DD0E0C930D1051CF06F2D18
:102F8000685C02C06F2D6F5C8FE796E00E94102B8B
:102F90008FE796E062EB79E00E94ED2ABE016F5F59
:102FA0007F4F8FE796E04AE050E00E94802C8FE749
:102FB00096E067EA79E00E94ED2A8E01095D1B4FD9
:102FC000D8011196EC91E032F8F48FE796E06AE9C7
:102FD00079E00E94ED2AF8018181803130F08FE79D
:102FE00096E063E371E00E94A72CC95DDB4F698125
:102FF00070E06F7070706F5F7F4F8FE796E04AE010
:1030000050E00E94932C0DC0F0E0EF70F070EE0FD6
:10301000FF1FE555FC4F608171818FE796E00E94AC
:10302000AA2CF39480913F05F81608F4A3CF8FE7FC
:1030300096E06FE779E00E94ED2A80913F040E94BC
:1030400048178FE796E064E679E00E94ED2A8091C8
:1030500040040E9448178FE796E069E479E00E94F7
:10306000ED2A809141040E9448178FE796E06EE2B6
:1030700079E00E94ED2A4091370450913804609124
:10308000390470913A04411551056105710539F112
:103090008FE796E02AE030E00E94E52B8FE796E08C
:1030A0006BEF78E00E94ED2A80913B040E94A0081B
:1030B000AB01BC018FE796E02AE030E00E94E52BEF
:1030C0008FE796E067ED78E00E94ED2A8FE796E0C3
:1030D00060913C044AE050E00E94302C06C08FE72B
:1030E00096E06EEC78E00E942E2B8FE796E061EB85
:1030F00078E00E94ED2A60913D0470913E048FE7D4
:1031000096E04AE050E00E940A2C8FE796E064E9DE
:1031100078E00E94ED2A60913604603150F470E04E
:103120006F5F7F4F8FE796E04AE050E00E94932C5C
:1031300006C08FE796E06BE878E00E942E2B8FE7C1
:1031400096E06EE678E00E94ED2A8091350480FDDD
:1031500003C065E371E002C069E371E08FE796E0C8
:103160000E94AA2C8FE796E061E578E00E94ED2AA4
:103170008091350482700E94180F8FE796E062E319
:1031800078E00E94ED2A8091350484700E94180F27
:103190008FE796E063E178E00E94ED2A80913504A4
:1031A00088700E94180FDF91CF911F910F91FF90AF
:1031B00008951F93CF93DF938FE796E062E57BE05E
:1031C0000E94ED2A4091020450910304609104048E
:1031D000709105048FE796E02AE030E00E94E52B2D
:1031E0008FE796E06CE37BE00E94ED2A40910604B5
:1031F0005091070460910804709109048FE796E0EC
:1032000020E130E00E94E52B8FE796E066E27BE06C
:103210000E94ED2A8FE796E060910A044AE050E0B0
:103220000E94302C8FE796E060E17BE00E94ED2A5F
:103230008FE796E060910B044AE050E00E94302C4A
:103240008FE796E06AEF7AE00E94ED2ACCE0D4E0C6
:1032500010E012C0112331F08FE796E06DE371E0CA
:103260000E94A72C8FE796E069914AE050E00E9407
:103270001E2C1F5F183119F08881882359F78FE7BA
:1032800096E00E94182B8FE796E064EE7AE00E94A9
:10329000ED2A8FE796E0609124044AE050E00E9416
:1032A000302C8FE796E06FEC7AE00E94ED2AE091F7
:1032B0002504F0E0E770F070EE0FFF1FE553FC4FC0
:1032C000608171818FE796E00E94AA2C8FE796E0DB
:1032D0006AEB7AE00E94ED2A8091250490E08871E3
:1032E00090708830910589F0893091051CF4892B04
:1032F00039F01BC08031910569F04897B1F40FC0D7
:103300008FE796E061EB7AE00EC08FE796E065EA22
:103310007AE009C08FE796E06FE97AE004C08FE7B2
:1033200096E065E97AE00E942E2B8FE796E061E84F
:103330007AE00E94ED2A4091FE035091FF036091D4
:103340000004709101048FE796E02AE030E00E94CB
:10335000E52B8FE796E068E67AE00E94ED2A8091FF
:10336000250480720E94180F8FE796E06FE47AE0E0
:103370000E94ED2A8091250480740E94180F8FE727
:1033800096E066E37AE00E94ED2A80912504807839
:103390000E94180F8FE796E069E17AE00E94ED2A1B
:1033A0008DEF93E00E94B008AB01BC018FE796E07F
:1033B0002AE030E00E94D62B8FE796E064E17AE0C5
:1033C0000E94ED2A8DEF93E00E94B0089B01AC01B2
:1033D00060E472E48FE090E00E94392F8FE796E07E
:1033E000BA01A9012AE030E00E94D62B8FE796E0CF
:1033F00061E17AE00E942E2BDF91CF911F91089519
:10340000EF92FF920F931F937C010FE716E0C80124
:103410006F2D70E04AE050E00E94F92BC8016EE287
:103420000E94102BB701E4E076956795EA95E1F7E5
:103430006F707070C8014AE050E00E94F92BC8011B
:103440006EE20E94102B8FE0E822FF24C801B70132
:103450004AE050E00E94F92B1F910F91FF90EF90EE
:1034600008950F931F93CF93DF932091B6042F3FBE
:10347000A9F58FE796E063E975E00E94ED2A84E5FF
:1034800093E00E94001A8FE796E062E775E00E94E1
:10349000ED2A80914005909141050E94001A8FE726
:1034A00096E06FE375E00E942E2B8FE796E06CE1CB
:1034B00075E00E942E2B8FE796E064E075E00E9495
:1034C0002E2B8FE796E06FED74E00E942E2B8FE796
:1034D00096E00E94182B0E94951769C012160CF0F6
:1034E00066C0332727FD309580913F0590E0821715
:1034F00093070CF45CC08FE796E06AEC74E00E94DE
:10350000ED2A6091B604772767FD70958FE796E006
:103510004AE050E00E94932C8FE796E06FE974E058
:103520000E94ED2A08E210E03AC0C12FD0E0CC0F93
:10353000DD1FC25EDA4F288130E08091B604992702
:1035400087FD909501972817390741F58FE796E099
:103550006FE371E00E94A72C8FE796E0602F4AE0AE
:1035600050E00E941E2C8FE796E063E471E00E9419
:10357000A72CE981F0E0EF70F070EE0FFF1FE5552A
:10358000FC4F608171818FE796E00E94A72C8FE746
:1035900096E067E471E00E94A72C0F5F1F5F8091A7
:1035A0003E05181710F28FE796E00E94182BDF9166
:1035B000CF911F910F910895CF92DF92EF92FF92DA
:1035C0000F931F93DF93CF93CDB7DEB76C970FB6F2
:1035D000F894DEBF0FBECDBF282F8091B6048F3F79
:1035E00009F050C1822F992787FD9095A92FB92FF7
:1035F000FC013A97EF36F10508F03DC1EC5CFF4F56
:10360000EE0FFF1F0590F491E02D09948FE796E0EF
:1036100069E471E0B4C08FE796E069E471E00E946C
:10362000AA2C22C18FE796E065E571E00E94AA2CE2
:1036300085E78983DE011296E7E2F4E08BE10190F1
:103640000D928150E1F7CE0101966CE10E94A50F29
:103650000E94340C83E08093FC0368EC70E080E00F
:1036600090E00E9493298091FC03843009F003C10B
:103670008FE70E94490A0E945D0A8983853509F017
:10368000FAC08FE796E061E874E00E942E2B8FE786
:1036900096E063E674E00E942E2B8FE796E065E4E7
:1036A00074E0B2C08FE796E06DE671E00E94AA2C4C
:1036B00089E68983CE01019661E00E94A50F0E94F0
:1036C000340C83E08093FC0368EC70E080E090E0D1
:1036D0000E9493298091FC03843009F0CCC08FE7CD
:1036E0000E94490A0E945D0A89838E010E5F1F4F66
:1036F0009DE1E92EF12CEC0EFD1E0E945D0AD80121
:103700008D938D01AE15BF05C1F7A7E2B4E0FE01B0
:1037100032968BE101900D928150E1F789818934D5
:1037200009F0A9C08FE796E067E274E00E942E2BB3
:103730008FE796E069E074E00E942E2B8FE796E019
:103740006BEE73E061C08FE796E067E871E00E947E
:10375000AA2C8EEF8093B6048EC020522750422FA1
:103760004053242F332727FD309580913F0590E06B
:10377000821793073CF48FE796E066E971E00E94B8
:10378000AA2C79C04093B6046FC084E18093B6043C
:103790008FE796E064EB73E037C085E18093B60471
:1037A0008FE796E06DE773E02FC086E18093B60463
:1037B0008FE796E066E473E027C087E18093B60464
:1037C0008FE796E06CEF72E01FC088E18093B6044B
:1037D0008FE796E06BEE72E017C089E18093B60444
:1037E0008FE796E067ED72E00FC08AE18093B60440
:1037F0008FE796E062EC72E007C08BE18093B6043D
:103800008FE796E06AE972E00E942E2B34C08FE7C2
:1038100096E060E872E00E942E2B8091350491E0E2
:103820001DC08FE796E06AE672E00E942E2B809121
:10383000350492E013C08FE796E065E572E00E94E0
:103840002E2B8091350494E009C08FE796E06AE35F
:1038500072E00E942E2B8091350498E08927809396
:1038600035048FEF8093B6040E94311A04C08FE7AD
:1038700096E00E943A2E8FE796E00E94002E892B58
:10388000B1F777C1822F0E948C16882309F471C189
:1038900080911C05882321F48FEF8093B60461C1C9
:1038A00087EB94E060E070E040E050E00E946E063C
:1038B0009B01AC019091B604963109F47CC097311C
:1038C00064F4943109F463C095310CF06AC0892F17
:1038D00081508D3008F035C113C0993109F4E5C02D
:1038E0009A313CF4973109F470C0983109F029C13C
:1038F000D2C09A3109F4E7C09B3109F022C1F5C06A
:10390000E92FFF27E7FDF09580913F0590E08E17A6
:103910009F070CF416C1DA01C9010197A109B10989
:103920008097A105B10540F0FF2410E008E26F0187
:103930000894C108D10826C0E95DFB4F822F815051
:103940008083E7C0612F70E0660F771F625E7A4F59
:10395000FB01808190E08C159D0599F4802F90E00B
:10396000A0E0B0E082179307A407B50749F4F60179
:10397000E95DFB4FDB0111968C918183FF24F39469
:103980000F5F1F5F80913E051817E0F2C0C02F3F08
:1039900031054105510511F008F0D3C020933F04D3
:1039A000B8C02F3F31054105510511F008F0C9C0DD
:1039B00020934004AEC02F3F31054105510511F061
:1039C00008F0BFC020934104A4C08091B704806276
:1039D000803719F588EB94E060E070E040E050E05B
:1039E0000E946E069B01AC01DC01CB010197A1098D
:1039F000B1090897A105B10508F0B6C0CA01B9011F
:103A000024ED30E340E050E00E94072F9B01AC0121
:103A10002A5E3C4A4A46554E24C0863611F588EB4C
:103A200094E060E070E040E050E00E946E069B0190
:103A3000AC01DC01CB010197A109B1090797A105F0
:103A4000B10508F091C0CA01B90128EA31E640E0A9
:103A500050E00E94072F9B01AC01245E3C434E4680
:103A6000544E211531054105510561F0DA01C901B6
:103A70008054914EAD49B8418158904FAA4FB24001
:103A800008F05FC020933704309338044093390422
:103A900050933A043EC02F3F31054105510511F0C6
:103AA00008F04FC020933B0434C0DA01C9010197EC
:103AB000A109B1098F3F9105A105B10508F041C0E9
:103AC00020933C0426C0DA01C901845C9940A040DF
:103AD000B0408D549D41A040B04038F430933E0436
:103AE00020933D04FF24F39401C0FF2421153105E8
:103AF0004105510511F48FEF07C021313105410512
:103B0000510528F4822F81508093360402C0FF2093
:103B1000C1F080911D058823D1F480910604909115
:103B20000704A0910804B09109040196A11DB11DDC
:103B30008093060490930704A0930804B0930904AB
:103B400006C08FE796E068EA71E00E94AA2C0E9406
:103B500082168FEF8093B6048FE796E06AE00E94AA
:103B6000422B0E94311A05C021E030E040E050E0D5
:103B70007DCF6C960FB6F894DEBF0FBECDBFCF9150
:103B8000DF911F910F91FF90EF90DF90CF900895FC
:103B90008FE796E06EEE71E00E942E2B8FE796E0A5
:103BA00066ED71E00E942E2B8FE796E00E94002EBA
:103BB000892B31F08FE796E00E943A2E0E94DC1AA2
:103BC0000E942C12823019F0833069F405C08FE70F
:103BD00096E068EB71E004C08FE796E061EA71E07F
:103BE0000E942E2B08958FEF8093B60410921D052E
:103BF0000E94311A0CC08FE796E00E94002E892B9C
:103C000031F08FE796E00E943A2E0E94DC1A8091F4
:103C1000B6048E3F81F708958091B604843009F48C
:103C20006FC0853084F4813009F45BC0823024F4A5
:103C30008F3F09F085C014C0823009F457C083302B
:103C400009F07EC058C0863009F464C086300CF498
:103C50005CC0873009F463C0893009F071C06AC064
:103C60008FE796E066E078E00E942E2B84E593E0F3
:103C70000E94001A8FE796E06EEE77E00E942E2BEE
:103C80008FE796E069EC77E00E942E2B8FE796E0B5
:103C90006FE977E00E942E2B8FE796E06EE777E0E2
:103CA0000E942E2B8FE796E061E577E00E942E2B95
:103CB0008FE796E06BE277E00E942E2B8FE796E08D
:103CC00067E077E00E942E2B8FE796E060EE76E0CB
:103CD0000E942E2B8FE796E00E94182B0E94D91885
:103CE0002FC08FE796E063EC76E028C08FE796E080
:103CF0006EE976E023C08FE796E069E876E01EC0C3
:103D00008FE796E06AE676E019C08FE796E066E214
:103D100076E014C08FE796E061E176E00FC08FE7B0
:103D200096E06CEF75E00E942E2B8FE796E066EB35
:103D300075E004C08FE796E060EA75E00E942E2BE4
:103D40006AE070E080E090E00E94932904C08FE771
:103D500096E00E943A2E8FE796E00E94002E892B73
:103D6000B1F708952F923F924F925F926F927F9298
:103D70008F929F92AF92BF92CF92DF92EF92FF927B
:103D80000F93DF93CF93CDB7DEB7A8970FB6F89414
:103D9000DEBF0FBECDBF7E010894E11CF11C80E1A7
:103DA000D7011D928A95E9F78FE796E066EC71E0FE
:103DB0000E94AA2C0E94F11220E431EE4DE958E154
:103DC00029A33AA34BA35CA380EC91EDA8E9BBE146
:103DD0008D8F9E8FAF8FB8A324EF31E040E050E08D
:103DE000298F3A8F4B8F5C8F30E5832E33EC932EE7
:103DF000A12CB12C80E491EEADE9B8E18D8B9E8BC6
:103E0000AF8BB88F44245524320100E022243324A0
:103E1000198A1A8A1B8A1C8A0DC18FE796E00E94B4
:103E20003A2E8434C9F0853434F48332C9F18C32AB
:103E300009F0CEC046C0833509F0CAC029A13AA115
:103E40004BA15CA1C901DA018D8B9E8BAF8BB88F22
:103E5000442455243201EEC08FE796E064E40E94CA
:103E6000102B8FE796E040E451EE6DE978E12AE00F
:103E700030E00E94442C8FE796E06CE20E94102B09
:103E80008FE796E040EC51ED68E97BE12AE030E015
:103E90000E94442C8FE796E06CE20E94422BCAC03D
:103EA00019821A821B821C821D821E821F82188622
:103EB00019861A861B861C861D861E861F86188AF2
:103EC0003CC00F5F043009F0B5C069817A818B81F5
:103ED0009C8128EE33E040E050E00E94072F69A368
:103EE0007AA38BA39CA36D817E818F8198850E948C
:103EF000072F6D8F7E8F8F8F98A329853A854B85ED
:103F00005C85298F3A8F4B8F5C8F6D857E858F8581
:103F1000988928EE33E040E050E00E94072F4B01E3
:103F20005C0160323EE4730730E0830730E09307C2
:103F300030F48CE162E30E94730A00E07BC06033DE
:103F400045E7740740E0840740E0940718F48CE1EB
:103F500062E2F1CF60345CE9750750E0850750E01C
:103F6000950718F48CE166E2E6CF80E5881683ECCD
:103F7000980680E0A80680E0B80618F48CE162E1BB
:103F8000DACF90E689169AEE990690E0A90690E0BD
:103F9000B90618F48CE165E1CECFA0E78A16A1E15D
:103FA0009A06A1E0AA06A0E0BA0618F48CE161E046
:103FB000C2CFB0EA8B16B6E89B06B1E0AB06B0E024
:103FC000BB0618F48CE163E0B6CF8CE165E0B3CFBB
:103FD00080538A3078F5C02EDD24CC0CDD1CCC0C4F
:103FE000DD1CE1E0F0E0EC0FFD1FCE0EDF1E282F00
:103FF000332727FD3095432F532F2DA33EA34FA3E7
:1040000058A7D6016D917D918D919C912AE030E069
:1040100040E050E00E94072F2DA13EA14FA158A5DE
:10402000260F371F481F591FD6012D933D934D93DF
:104030005C9313978FE796E00E94002E892B09F07E
:10404000ECCE411451046104710499F46D897E89A8
:104050008F89988D0E94E90A61E070E080E090E02D
:104060000E94932922242A943324198A1A8A1B8AAB
:104070001C8A298D3A8D4B8D5C8D42165306640641
:104080007506D0F40E94940A29893A894B895C8983
:10409000280F311D411D511D298B3A8B4B8B5C8B99
:1040A000381608F4382E821508F4282E0894411C7E
:1040B000511C611C711C64C06D897E898F89988D2B
:1040C00028EE33E040E050E00E94392F8FE796E081
:1040D000BA01A9012AE030E00E94D62B8FE796E0D2
:1040E0006CE20E94102B8FE796E0632D4AE050E0CF
:1040F0000E941E2C8FE796E06CE20E94102B6989CB
:104100007A898B899C89A30192010E94392F8FE7BC
:1041100096E0BA01A9012AE030E00E94D62B8FE791
:1041200096E06CE20E94102B8FE796E0622D4AE049
:1041300050E00E941E2C8FE796E06CE20E94422B1A
:104140008D899E89AF89B88D880D991DAA1DBB1DCB
:104150008D8B9E8BAF8BB88F2D8D3E8D4F8D58A143
:10416000281739074A075B0740F489A19AA1ABA138
:10417000BCA18D8B9E8BAF8BB88F4424552432010C
:1041800029A13AA14BA15CA1285E33404040504098
:1041900009F050CFA8960FB6F894DEBF0FBECDBF82
:1041A000CF91DF910F91FF90EF90DF90CF90BF9074
:1041B000AF909F908F907F906F905F904F903F90C7
:1041C0002F900895CF92DF92EF92FF920F931F935B
:1041D000DF93CF93CDB7DEB7E8970FB6F894DEBF85
:1041E0000FBECDBF7C01FC018281883009F4ABC0D9
:1041F0008930A8F4843009F45FC0853048F48230F7
:10420000E9F1833008F04DC0813009F080C123C04E
:10421000863009F482C0873008F08BC060C08836D1
:1042200009F4D4C0893650F4863609F4AFC0873615
:1042300008F0C5C0853609F06AC18FC08A3609F416
:10424000FEC08A3608F4F2C08B3609F438C1873CC8
:1042500009F05DC149C1C70161E049E250E00E9437
:1042600079110DEF13E0C701F80161918F010E94F0
:104270005911F4E006321F07B1F753C1C70162E0DC
:104280004BE150E00E94791107E214E0C701F80108
:1042900061918F010E945911F4E002341F07B1F7B8
:1042A00040C1C70163E041E050E00E9479110E94E3
:1042B0002C12682FC70133C1C70164E041E050E010
:1042C0000E947911C70161E00E9459118FE796E0C1
:1042D000F70164810E94732E0E94B21E28C1409192
:1042E0003E0550E0440F551FC70165E00E9479115B
:1042F00000E010E009C0F801E25EFA4FC7016081FA
:104300000E9459110F5F1F4F80913E0590E0880F6A
:10431000991F0817190778F304C1C70166E042E046
:1043200050E00E947911C70164E573E00E946A11B0
:10433000F8C0C70167E041E050E00E947911C70171
:1043400060913F05ECC0C70168E041E050E00E9489
:104350007911C70160912604E2C0C70165E641E01A
:1043600050E00E947911F70187819085899709F0C3
:10437000D4C0D701EDEFF3E019968C911997819392
:10438000119684E0E632F807B9F7ABC0C70166E6DC
:1043900041E050E00E947911F701878190854B97A9
:1043A00009F0BBC0D701E7E2F4E019968C911997A8
:1043B0008193119684E0E234F807B9F792C0C701FF
:1043C00067E641E050E00E94791189C0C70168E6C4
:1043D00041E050E00E94791185E78983DE01129661
:1043E000E7E2F4E08BE101900D928150E1F7CE011C
:1043F00001966CE10E94A50F0E94340C83E080932B
:10440000FC0368EC70E080E090E00E9493298091CA
:10441000FC03843009F081C08FE70E94490A0E94A2
:104420005D0A8983853509F078C05BC0C70169E6FC
:1044300041E050E00E9479110E94280852C0C70153
:104440006AE641E050E00E94791189E68D8FCE0145
:104450004D9661E00E94A50F0E94340C83E080938A
:10446000FC0368EC70E080E090E00E94932980916A
:10447000FC03843009F051C08FE70E94490A0E9472
:104480005D0A8D8F8E01025E1F4F49E3C42ED12C31
:10449000CC0EDD1E0E945D0AF80181938F01EC15A0
:1044A000FD05C1F7A7E2B4E0FE017E968BE1019025
:1044B0000D928150E1F78D8D893479F512C0C701D5
:1044C0006BE641E050E00E947911F70181850E947E
:1044D000B5130E94D807892B21F40E9428080E9456
:1044E0004A13C70161E01BC0C70167EC41E050E01F
:1044F0000E947911C70161E00E9459118FE796E08F
:10450000F70164810E94732E1092480410C0C70105
:104510006AEC41E050E00E947911C70160E00E941E
:1045200059118FE796E0F70164810E94732EE89697
:104530000FB6F894DEBF0FBECDBFCF91DF911F91B4
:104540000F91FF90EF90DF90CF9008956F927F9240
:104550008F929F92AF92BF92CF92DF92EF92FF9293
:104560000F931F93CF93DF9381E0809348048EE4F1
:10457000E82E84E0F82E04E0C02ED12CCE0CDF1CF7
:1045800014E6612EB4E07B2EA6E09A2EF5E08F2E85
:10459000E2E0AE2E73E0B72EB8C08FE796E00E943F
:1045A000002E892B09F4B1C0A9C08FE796E00E94C4
:1045B0003A2E982F8093490480914A04833021F148
:1045C000843028F4813099F08230B8F409C0853005
:1045D00009F450C0853020F1863009F08FC067C0E3
:1045E000953B09F08BC081E080934A0487C09236E6
:1045F00009F082C0A0924A0481C090934B0490932A
:104600004C04B0924A047AC090934E04F701118290
:1046100080914C04892780934C0470924A046EC0A8
:10462000D92FC0E020914E0430914F042C2B3D2B0C
:1046300030934F0420934E0480914C04892780933B
:104640004C0480924A042536310508F457C089E4A9
:1046500094E06CEC41E050E00E94791189E494E030
:1046600061E00E9459118FE796E060914D040E942D
:10467000732E42C02091500430915104F901E75B40
:10468000FB4F918780914C04892780934C042F5FC6
:104690003F4F309351042093500480914E049091E9
:1046A0004F042817390750F190924A0427C000910F
:1046B0004C04091729F489E494E00E94E22013C015
:1046C00010914B0489E494E06BEC42E050E00E94CE
:1046D000791189E494E0612F0E94591189E494E0F2
:1046E000602F0E945911F601862D11928A95E9F7E3
:1046F000109251041092500410924A048FE796E0F1
:104700000E94002E892B09F050CF809148048130FF
:1047100009F443CFDF91CF911F910F91FF90EF905C
:10472000DF90CF90BF90AF909F908F907F906F90D1
:104730000895DF92EF92FF920F931F93CF93DF9331
:104740000E946D296115710581059105C9F30E94CB
:104750006506109206041092070410920804109245
:104760000904DD24E0900604F09007040091080499
:1047700010910904102F0F2DFE2CEE240E946006CC
:104780002FEF30E040E050E00E945B2FE60EF71E76
:10479000081F191FE0920604F09207040093080412
:1047A00010930904D39484E0D816E1F6CCE0D4E069
:1047B00010E017C00E94600622E330E040E050E0C5
:1047C0000E945B2F6F5FECE0F4E090E004C0819109
:1047D000861781F39F5F9117D0F369931F5F18319C
:1047E00019F08881882331F7DF91CF911F910F91C4
:1047F000FF90EF90DF9008951F931091B6041F3F34
:1048000009F0BFC0893409F466C08A342CF58833B6
:1048100009F476C089336CF4803309F481C08133A4
:104820000CF06CC08B3109F44CC0813209F0A3C08C
:104830003CC0813409F483C082343CF4893309F4E8
:104840006DC0803409F097C030C0823409F482C052
:10485000863409F090C04FC0823609F47BC083369D
:104860008CF4883571F1893534F48235E9F183357A
:1048700009F081C01FC08A3509F478C0813609F07B
:104880007AC05DC0823781F1833734F4863699F17E
:10489000893609F070C01FC0883799F08A3709F44B
:1048A00065C0833709F067C005C08FE796E069E40B
:1048B00071E017C00E944A138FE796E063ED71E044
:1048C00006C00E94D8078FE796E06DEE71E00E9467
:1048D000AA2C8EEF4EC00E9428088FE796E06CE06D
:1048E00072E00E94AA2C47C00E9499238FE796E0AD
:1048F00065E272E0F6CF0E94FF163DC0805339C0DA
:104900008FE796E06EE871E00E942E2B90912504CF
:10491000892F885F8871977E892B0CC089E029C018
:104920008FE796E06BE771E00E942E2B80912504C3
:1049300090E28927809325041093B6041CC08FE76A
:1049400096E065E671E00E942E2B8091250490E4AC
:10495000892709C08FE796E064E571E00E942E2B5D
:104960008091250480588093250402C00E94C81DB0
:104970008FEF8093B6048091B6048E3F09F4E8C0AF
:10498000DFC00E948C16882309F4E2C080911C05C8
:10499000882321F48FEF8093B604D2C087EB94E094
:1049A00060E070E040E050E00E946E069B01AC01C8
:1049B0008091B604843009F441C0853044F48230DB
:1049C00041F1833094F5813009F096C00DC08630F6
:1049D00009F467C086300CF43EC0873009F469C022
:1049E000893009F089C075C0DA01C9018154914E3E
:1049F000AD49B8418F57904FAA4FB24008F07CC0E4
:104A0000209302043093030440930404509305045C
:104A10009AC02093060430930704409308045093EF
:104A2000090481E080931D058EC0283031054105C1
:104A3000510508F061C020930A0485C0DA01C9015C
:104A40000197A109B1090A97A105B10508F054C061
:104A500020930B0478C087EB94E06DE371E00E9433
:104A60008A0710E00EC0183130F4E12FF0E0E35077
:104A7000FC4F87871F5F80E090E06DE371E00E944C
:104A80008A07009759F00E946C07009761F706C0EB
:104A9000E12FF0E0E350FC4F17861F5F1831C0F3A1
:104AA00052C0253031054105510530F520932404CD
:104AB0004AC0DA01C9010197A109B1090697A10508
:104AC000B105D0F480912504887F822B8093250442
:104AD0003AC0DA01C9010197A109B1098050924C8D
:104AE000A140B04048F42093FE033093FF0340936D
:104AF00000045093010427C08FE796E068EA71E054
:104B00000E94AA2C13C08091060490910704A091E2
:104B10000804B09109040196A11DB11D80930604FB
:104B200090930704A0930804B09309040E9482168E
:104B30008FEF8093B6048FE796E06AE00E94422BE5
:104B40000E940C1E05C080911D058823E1F2EECF66
:104B50001F9108958FEF8093B60410921D050E9457
:104B60000C1E0CC08FE796E00E94002E892B31F0BE
:104B70008FE796E00E943A2E0E94FC238091B604B3
:104B80008E3F81F76AE070E080E090E00E94932918
:104B900004C08FE796E00E943A2E8FE796E00E94CD
:104BA000002E892BB1F708957F928F929F92AF923A
:104BB000BF92CF92DF92EF92FF920F931F93DF93FA
:104BC000CF93CDB7DEB7AA970FB6F894DEBF0FBE6E
:104BD000CDBF0E945F296B017C0181E00E94550BD3
:104BE00004C08FE796E00E943A2E8FE796E00E947D
:104BF000002E892BB1F75E98409811E032E6732EB3
:104C000022E0822E912C8C0E9D1E5E010894A11C28
:104C1000B11C03E00E945F2920E030E06C197D099F
:104C20008E099F09693C71058105910510F021E00D
:104C300030E0812F90E028233923232BB9F10E9403
:104C40005F296B017C015D9A419A80ED97E00E949B
:104C5000B4117982D401EDEFF3E089E201900D9275
:104C60008150E1F7C5016AE20E94A50F5D98419865
:104C700080E090E00E94B4110093FC030E94340C89
:104C800062E370E080E090E00E9493298091FC0351
:104C9000843059F40093FC038FE70E94490A0E9474
:104CA0005D0A823411F410E001C011E082E10E943B
:104CB000932A892B61F511E02AC05E9A409A5D9A89
:104CC000419A8FE796E00E943A2E8D30910569F067
:104CD0008E3091051CF40A97B1F407C08332910518
:104CE00069F08234910579F40CC08FE796E066E4B0
:104CF00071E00E942E2B0E94AA2505C00E94B21EC0
:104D000002C00E94A6225E9840985D9841988FE765
:104D100096E00E94002E892B09F47CCFCECF8FE73E
:104D200096E00E94002E04970CF18FE796E00E9417
:104D30003A2E82349105D1F48FE796E00E943A2E04
:104D40008E34910599F48FE796E00E943A2E8434D0
:104D5000910561F48FE796E00E943A2E819731F435
:104D600080E090E00E94B4110E94D42508958F92B3
:104D70009F92AF92BF92CF92DF92EF92FF920F93EA
:104D80001F9382E10E94932A892B09F0ACC068EC42
:104D900070E080E090E00E94932980E090E00E9423
:104DA000B4110E945F295B016C0140ECE42E42E1EA
:104DB000F42E012D112DE60EF71E081F191F06C037
:104DC00082E10E94932A892B09F085C00E945F2905
:104DD0006E157F058007910798F382E10E94932A60
:104DE000892B09F078C080ED97E00E94B4110E94F1
:104DF0005F297B018C0199249394882488E496E2AE
:104E0000A0E0B0E0A80EB91ECA1EDB1E29C0AE1479
:104E1000BF04C006D10638F480ED97E00E94B411BB
:104E2000882483941DC00E945F296E197F09800B1E
:104E3000910B693C71058105910590F00E945F29F5
:104E40007B018C0180E0992009F481E0982E882371
:104E500019F480E090E002C080ED97E00E94B41168
:104E600082E10E94932A892B91F280E090E00E94D7
:104E7000B411882051F1809126048F5F83700E94C5
:104E8000B5138FE796E062E472E00E94A72C8FE7EB
:104E900096E0609126044AE050E00E94302C0E9487
:104EA000D807892B39F08FE796E06FE472E00E9413
:104EB000AA2C19C08FE796E06CE672E00E94A72C3E
:104EC0000E9428080E944A130EC00E9499230E9443
:104ED0004A130E94D9188FE796E06EE872E00E94AC
:104EE000AA2C0E94D4251F910F91FF90EF90DF9084
:104EF000CF90BF90AF909F908F90089580E069EC25
:104F000077E042E050E00E949A280895EF92FF92E5
:104F10000F931F930E949F1186E061E00E94F42985
:104F200085E061E00E94F4298EE061E00E94F429AE
:104F30008FE061E00E94F42982E160E00E94F429A0
:104F400088E060E00E94F42988E061E00E94602A25
:104F50000E94F6118FE796E040E052EC61E070E0CD
:104F60000E94792D0E94A4130E94D807892B39F042
:104F70008FE796E06FE472E00E94AA2C0AC08FE7E8
:104F800096E06CE672E00E94A72C0E9428080E941E
:104F90004A130E94F90C8FEF809373050E947E27BD
:104FA00078940E945F297B018C01809173058F3F6B
:104FB00009F0B0C00E945F296E197F09800B910B28
:104FC000605D77408040904008F0A4C0EECF8FE74E
:104FD00096E00E943A2E8FE796E00E94002E892BE1
:104FE000B1F78FE796E065EA72E00E94A72C84E5AE
:104FF00093E00E94001A8FE796E06CEB72E00E944B
:10500000A72C8FE796E065E070E04AE050E00E9450
:10501000932C68EC70E080E090E00E9493290E945D
:105020008F264091FE035091FF0360910004709120
:105030000104DB01CA010197A109B1090497A10587
:10504000B10568F440937405433029F040E052EC18
:1050500061E070E004C040EA56E861E070E08FE78C
:1050600096E00E94792D0E94B7265E98409880E0D5
:1050700090E00E94B4110E94F90C80E00E94550B50
:10508000809159050E947E0A0E94340C1092DE0520
:105090001092DF051092E0056CE271E080E090E094
:1050A0000E94932980ED97E00E94B41164E670E0BD
:1050B00080E090E00E94932980E090E00E94B4118B
:1050C00010E015C064E670E080E090E00E94932953
:1050D00080ED97E00E94B41164E670E080E090E01B
:1050E0000E94932980E090E00E94B4111F5F80919C
:1050F0002604181738F38091250490E084FF15C02A
:1051000020E088719070489709F421E0822F0E9476
:105110000D120BC080ED97E00E94B41182E161E0B6
:105120000E94602A5E9A409A56CF1F910F91FF907D
:10513000EF900895823000F5E82FF0E0EE0FFF1FAA
:10514000E651FA4F71836083882319F08130A1F40E
:1051500008C0809169008C7F842B80936900E89A55
:10516000089580916900440F551F440F551F837F98
:10517000842B80936900E99A08951F920F920FB6CD
:105180000F9211242F933F934F935F936F937F93CD
:105190008F939F93AF93BF93EF93FF938091EA0513
:1051A0009091EB05892B29F0E091EA05F091EB0550
:1051B0000995FF91EF91BF91AF919F918F917F9151
:1051C0006F915F914F913F912F910F900FBE0F9074
:1051D0001F9018951F920F920FB60F9211242F93C4
:1051E0003F934F935F936F937F938F939F93AF936F
:1051F000BF93EF93FF938091EC059091ED05892B80
:1052000029F0E091EC05F091ED050995FF91EF9102
:10521000BF91AF919F918F917F916F915F914F91CE
:105220003F912F910F900FBE0F901F9018951F92D6
:105230000F920FB60F9211242F933F938F939F934A
:10524000AF93BF938091F2059091F305A091F4057F
:10525000B091F5053091F6050196A11DB11D232FE2
:105260002D5F2D3720F02D570196A11DB11D2093E4
:10527000F6058093F2059093F305A093F405B0939F
:10528000F5058091EE059091EF05A091F005B091A4
:10529000F1050196A11DB11D8093EE059093EF05D8
:1052A000A093F005B093F105BF91AF919F918F91BD
:1052B0003F912F910F900FBE0F901F9018958FB7B1
:1052C000F8942091F2053091F3054091F405509146
:1052D000F5058FBFB901CA0108959FB7F8942091D1
:1052E000EE053091EF054091F0055091F10586B53E
:1052F000A89B06C08F3F21F02F5F3F4F4F4F5F4F5E
:105300009FBF542F432F322F2227280F311D411DBD
:10531000511D82E0220F331F441F551F8A95D1F77C
:10532000B901CA010895EF92FF920F931F93CF9393
:10533000DF937B018C010E946D29EB010EC00E945E
:105340006D296C1B7D0B685E7340C8F30894E108FF
:10535000F10801091109C851DC4FE114F1040105FC
:10536000110569F7DF91CF911F910F91FF90EF9099
:105370000895789484B5826084BD84B5816084BDCD
:1053800085B5826085BD85B5816085BDEEE6F0E0BE
:10539000808181608083E1E8F0E01082808182601A
:1053A0008083808181608083E0E8F0E0808181609B
:1053B0008083E1EBF0E0808184608083E0EBF0E0CB
:1053C000808181608083EAE7F0E08081846080836F
:1053D0008081826080838081816080838081806819
:1053E00080831092C1000895CF93DF93482F50E03F
:1053F000CA018656944FFC0134914A57544FFA0122
:105400008491882369F190E0880F991FFC01E85985
:10541000F44FA591B491FC01EE58F44FC591D4918D
:10542000662351F42FB7F8948C91932F909589238C
:105430008C93888189230BC0623061F42FB7F89474
:105440008C91932F909589238C938881832B8883CB
:105450002FBF06C09FB7F8948C91832B8C939FBF6E
:10546000DF91CF910895833071F0843028F481303A
:10547000A1F0823021F514C08630B1F08730D1F030
:105480008430E9F404C0809180008F7703C080915C
:1054900080008F7D80938000089584B58F7702C04F
:1054A00084B58F7D84BD08958091B0008F778093FF
:1054B000B00008958091B0008F7D8093B000089572
:1054C000FF920F931F93F62E482F50E0CA0182558A
:1054D000944FFC012491CA018656944FFC0114910B
:1054E0004A57544FFA0104910023C9F0222319F0BE
:1054F000822F0E94332AE02FF0E0EE0FFF1FEE58BC
:10550000F44FA591B4919FB7F894FF2021F48C91AA
:105510001095812302C08C91812B8C939FBF1F918A
:105520000F91FF9008950F931F93482F50E0CA01E9
:105530008255944FFC012491CA018656944FFC0178
:1055400004914A57544FFA011491112319F420E0A1
:1055500030E015C0222319F0822F0E94332A812FB8
:1055600090E0880F991F8458944FFC01A591B49145
:105570008C9120E030E0802311F021E030E0C9017F
:105580001F910F910895CF92DF92EF92FF920F93A8
:105590001F93CF93DF937C016B018A01C0E0D0E0C1
:1055A0000FC0D6016D916D01D701ED91FC91019075
:1055B000F081E02DC7010995C80FD91F0150104097
:1055C0000115110571F7CE01DF91CF911F910F9158
:1055D000FF90EF90DF90CF900895EF92FF920F939E
:1055E0001F93CF93DF937C018B01C0E0D0E0F801E3
:1055F0000F5F1F4F6491662359F0D701ED91FC9125
:105600000190F081E02DC7010995C80FD91FEFCF98
:10561000CE01DF91CF911F910F91FF90EF900895F0
:10562000DC01ED91FC910190F081E02D0995089548
:10563000EF92FF920F931F938C016DE00E94102B4D
:105640007C01C8016AE00E94102B9C012E0D3F1DB9
:10565000C9011F910F91FF90EF900895EF92FF9273
:105660000F931F937C010E94ED2A8C01C7010E94B9
:10567000182B9C01200F311FC9011F910F91FF9022
:10568000EF900895EF92FF920F931F937C010E9479
:10569000102B8C01C7010E94182B9C01200F311F79
:1056A000C9011F910F91FF90EF900895CF93DF9361
:1056B000EC016115710519F420E030E00FC0DB0149
:1056C0000D900020E9F71197A61BB70BE881F9812F
:1056D0000280F381E02DAD0109959C01C901DF91A4
:1056E000CF9108954F925F927F928F929F92AF9247
:1056F000BF92CF92DF92EF92FF920F931F93DF93AF
:10570000CF93CDB7DEB7A1970FB6F894DEBF0FBE2B
:10571000CDBF2C01742ECB01223008F42AE019A24F
:1057200031E2C32ED12CCC0EDD1E822E9924AA2468
:10573000BB24672D752FA50194010E94392F790193
:105740008A01C801B701A50194010E94072F472DC6
:10575000461B0894C108D1084A3014F4405D01C0CA
:10576000495CF6014083E114F1040105110521F0C3
:105770007E2C5F2DC801DDCFC201B6010E94562BE1
:10578000A1960FB6F894DEBF0FBECDBFCF91DF91CB
:105790001F910F91FF90EF90DF90CF90BF90AF904F
:1057A0009F908F907F905F904F900895DC0121151E
:1057B000310541F4ED91FC910190F081E02D642FD1
:1057C000099508950E94722B0895EF92FF920F930E
:1057D0001F937C010E94D62B8C01C7010E94182BBD
:1057E0009C01200F311FC9011F910F91FF90EF9075
:1057F0000895EF92FF920F931F939A017B0100E0AF
:1058000010E0B801A7010E94D62B1F910F91FF90C5
:10581000EF900895EF92FF920F931F937C010E94E7
:10582000F92B8C01C7010E94182B9C01200F311FFE
:10583000C9011F910F91FF90EF900895EF92FF9291
:105840000F931F939A01E62EFF2400E010E0B801A9
:10585000A7010E94D62B1F910F91FF90EF90089502
:10586000EF92FF920F931F937C010E941E2C8C01DC
:10587000C7010E94182B9C01200F311FC9011F91E5
:105880000F91FF90EF900895CF92DF92EF92FF92E9
:105890000F931F93CF93DF93EC016A017B012115D6
:1058A000310541F4E881F9810190F081E02D642F08
:1058B00009951BC02A303105B1F477FF13C06DE2A2
:1058C0000E94102B8C0144275527BA014C195D0901
:1058D0006E097F09CE012AE00E94722B9C01200FE5
:1058E000311F04C02AE00E94722B9C01C901DF9184
:1058F000CF911F910F91FF90EF90DF90CF9008957F
:10590000EF92FF920F931F937B019A010027F7FC00
:105910000095102FB801A7010E94442C1F910F91F0
:10592000FF90EF900895EF92FF920F931F937C01E9
:105930000E94802C8C01C7010E94182B9C01200F13
:10594000311FC9011F910F91FF90EF9008950E94A0
:10595000562B0895EF92FF920F931F937C010E94A4
:10596000A72C8C01C7010E94182B9C01200F311F0E
:10597000C9011F910F91FF90EF90089508951F9214
:105980000F920FB60F9211242F933F934F938F9343
:105990009F93EF93FF938091C00082FD1DC04091C3
:1059A000C60020913706309138062F5F3F4F2F7386
:1059B00030708091390690913A062817390771F0B6
:1059C000E0913706F0913806E950FA4F4083309362
:1059D00038062093370602C08091C600FF91EF91F0
:1059E0009F918F914F913F912F910F900FBE0F90EC
:1059F0001F9018951F920F920FB60F9211242F939C
:105A00003F938F939F93EF93FF9320917B06309169
:105A10007C0680917D0690917E062817390731F427
:105A20008091C1008F7D8093C10014C0E0917D06FC
:105A3000F0917E06E55CF94F208180917D06909182
:105A40007E0601968F73907090937E0680937D06FC
:105A50002093C600FF91EF919F918F913F912F91DD
:105A60000F900FBE0F901F9018958F929F92AF923C
:105A7000BF92CF92DF92EF92FF920F931F93DF932B
:105A8000CF93CDB7DEB7FC011382128288EE93E08C
:105A9000A0E0B0E084839583A683B7838DEE93E086
:105AA000918380837587648757874687318B208BE6
:105AB000138B028BF58AE48AD78AC68AB18EA08EB0
:105AC000938E828E8F85848F8889858F8989868F32
:105AD0008A89878F8B8980A3CF91DF911F910F9146
:105AE000FF90EF90DF90CF90BF90AF909F908F90FE
:105AF0000895AF92BF92DF92EF92FF920F931F93A0
:105B0000CF93DF93EC017A018B01DD24403081EEED
:105B1000580780E0680780E0780711F0DD24D3940F
:105B200091E0A92EB12CEC89FD89DD2069F0C50139
:105B300008A002C0880F991F0A94E2F7808360E0F2
:105B400079E08DE390E005C0108260E874E88EE1B2
:105B500090E0A80197010E94392F21503040404029
:105B60005040569547953795279580E12030380766
:105B700020F0DD2011F0DD24D6CFE889F9893083CB
:105B8000EA89FB89208319A2EE89FF89408121E0FF
:105B900030E0C9010C8C02C0880F991F0A94E2F70B
:105BA000482B4083EE89FF894081C9010D8C02C0DA
:105BB000880F991F0A94E2F7482B4083EE89FF89EA
:105BC0004081C9010E8C02C0880F991F0A94E2F728
:105BD000482B4083EE89FF8980810F8C02C0220F01
:105BE000331F0A94E2F7209528232083DF91CF9179
:105BF0001F910F91FF90EF90DF90BF90AF900895AD
:105C0000DC011C96ED91FC911D97E05CFF4F21910A
:105C1000319180819181281B390B2F733070C9011C
:105C200008958FE796E00E94002E892B11F00E94C4
:105C3000BE2C0895DC011C96ED91FC911D97E05C53
:105C4000FF4F20813181E054F040DF01AE5BBF4F58
:105C50008D919C9111972817390719F42FEF3FEF79
:105C600007C08D919C91E80FF91F8081282F30E0AB
:105C7000C9010895DC011C96ED91FC911D97E05C33
:105C8000FF4F20813181E054F040DF01AE5BBF4F18
:105C90008D919C9111972817390719F42FEF3FEF39
:105CA00010C08D919C911197E80FF91F20818D9163
:105CB0009C91119701968F73907011969C938E937F
:105CC00030E0C9010895DC0191968C919197882369
:105CD00039F05496ED91FC915597808186FFF9CF6C
:105CE00091961C920895CF93DF93EC01EE85FF858A
:105CF000E05CFF4F20813181E054F0402F5F3F4F47
:105D00002F733070DF01AE5BBF4F8D919C91119767
:105D100028173907D1F3E05CFF4F80819181E0546F
:105D2000F040E80FF91F6083EE85FF85E05CFF4FD0
:105D300031832083EE89FF89208181E090E00F8C00
:105D400002C0880F991F0A94E2F7282B208381E074
:105D500089A3EC89FD8980818064808381E090E063
:105D6000DF91CF9108958F929F92AF92BF92CF9281
:105D7000DF92EF92FF920F931F9300D000D00F920B
:105D8000EDB7FEB7319684E0ADB7BEB711968C93F0
:105D900083E0818387E0828385E0838381E084835D
:105DA0008FE796E067EF75E04BE356E025EC30E0D7
:105DB00004EC10E0B0ECEB2EF12CA1ECCA2ED12CAF
:105DC000F2ECAF2EB12CE6EC8E2E912C0E94352DEC
:105DD0000F900F900F900F900F901F910F91FF90C9
:105DE000EF90DF90CF90BF90AF909F908F900895ED
:105DF000CF93DF930E94B9290E948627C1E1DEE29A
:105E00000E9412142097E1F30E94112EF9CF629F95
:105E1000D001739FF001829FE00DF11D649FE00DA2
:105E2000F11D929FF00D839FF00D749FF00D659F03
:105E3000F00D9927729FB00DE11DF91F639FB00D02
:105E4000E11DF91FBD01CF011124089597FB092E13
:105E500007260AD077FD04D049D006D000201AF4D6
:105E6000709561957F4F0895F6F7909581959F4FB6
:105E70000895A1E21A2EAA1BBB1BFD010DC0AA1F8B
:105E8000BB1FEE1FFF1FA217B307E407F50720F0A3
:105E9000A21BB30BE40BF50B661F771F881F991F1E
:105EA0001A9469F760957095809590959B01AC0167
:105EB000BD01CF01089597FB092E05260ED057FD91
:105EC00004D0D7DF0AD0001C38F4509540953095A7
:105ED00021953F4F4F4F5F4F0895F6F7909580956E
:105EE000709561957F4F8F4F9F4F0895AA1BBB1BE5
:105EF00051E107C0AA1FBB1FA617B70710F0A61BCA
:105F0000B70B881F991F5A95A9F780959095BC01EA
:105F1000CD010895EE0FFF1F0590F491E02D099437
:105F2000911106C0803219F089508550D0F708953C
:105F30009927882708952F923F924F925F926F92F0
:105F40007F928F929F92AF92BF92CF92DF92EF9209
:105F5000FF920F931F93CF93DF93CDB7DEB7CA1B8A
:105F6000DB0B0FB6F894DEBF0FBECDBF09942A88B5
:105F7000398848885F846E847D848C849B84AA845D
:105F8000B984C884DF80EE80FD800C811B81AA81EA
:105F9000B981CE0FD11D0FB6F894DEBF0FBECDBFB5
:085FA000ED010895F894FFCF14
:105FA8004E6F005965730054582074696D656F759C
:105FB8007421006D6F64756C65206C6F636B65642C
:105FC8003F00486F70206368616E6E656C2000202A
:105FD80040200053004E2F4100386368002C002CED
:105FE800205B005D20280029004E4F5420454E417B
:105FF800424C45440053656E64696E67207365744E
:1060080074696E677320746F2052580A0052657362
:10601800657474696E672073657474696E6773203C
:106028006F6E2052580A0041626F72746564206571
:10603800646974730A00696E76616C6964207365BB
:106048006C656374696F6E000D0A496E76616C69E0
:106058006420696E707574202D20646973636172A1
:106068006465642107007363616E6E6572206D6FED
:1060780064650053657474696E677320736176652F
:106088006420746F20454550524F4D0A0052657682
:1060980065727465642073657474696E67732066CD
:1060A800726F6D20454550524F4D0A004C6F616428
:1060B800656420666163746F7279206465666175D2
:1060C8006C74730A004B657920616E6420636861A3
:1060D8006E6E656C732072616E646F6D697A65644B
:1060E8000A004E65772070726F66696C653A004CDD
:1060F8006F616465642073657474696E6773206684
:10610800726F6D20454550524F4D0A00454550521B
:106118004F4D2064617461206E6F742076616C69E4
:10612800642C207265696E6974696E670A00456E31
:10613800746572696E672062696E64696E67206D46
:106148006F64650A004F70656E4C52536E67205439
:1061580058207374617274696E672000206F6E2016
:106168004857200050504D00525353490053444162
:106178000053434C00525844005458440041494E7F
:10618800004C424545500053504B54524D00534229
:1061980055530053554D44004C4C494E440000346F
:1061A8002B34003800382B340031320031322B3494
:1061B8000031360001000000C01200001A400AA198
:1061C800204EA5001B1E27522C23308025000005D9
:1061D800400AA1204EA50020244EA52C2330004BB8
:1061E800000006400AD0009D49007B289D492C23C9
:1061F8003000E1000005400A4501D7DC03B81E0E57
:10620800BF00232E48E801008A400A600155550264
:10621800AD1E20000023C88025000005400AA120EB
:106228004EA50020244EA52C2330000200020002B7
:106238000002000200020002000200020002000246
:1062480000020002000200020002FFC402C802CDE0
:1062580002D102D502D902DD02E102E702EE02F321
:1062680002F802FE02FE02FE02FE023501FF0203F0
:1062780003050309030C031103350100070B0C1078
:10628800111500160A1322312900000000732EC3CD
:0A6298002A002E3A2E1A2E632E0063
:00000001FF
